:1000000012C0189518951895189518951895189563
:100010004FC4189518958ACA18951895189518956B
:100020001895189518958FE58DBFC0E4E8EB4E2E16
:1000300084E08EBFD4E0F3E05F2EA89584B7082E4D
:10004000877F84BF88E1992781BD91BDEEEFF3E002
:10005000A0E6B0E088278D933197E9F783E389B96B
:1000600080E080BD88E18AB9662480E08FBD84E0AD
:100070008EBD8EEE95E89DBD8CBD79B7746079BF5D
:100080008C9A8F9ABB9ABD9A8D9A12D911D94ED952
:10009000ECE5FAE0A3E3B3E0ED93FC93A09A579A62
:1000A000A89A00E010E020E030E0A5EEB2E00D9369
:1000B0001D932D933C9381E080936000009160003C
:1000C0000C3310F009F011C080E0A0E6B0E0AD9074
:1000D000BB24A2EFB2E0AA0DBB1D8C93A0E6B0E05A
:1000E0008C918F5F8C9308F4E9CF81E090E0A2E6D9
:1000F000B0E08D939C93A2E6B0E00D911C9100308E
:1001000052E0150710F009F00FC080E0A2E6B0E061
:10011000AD90BD90A3E6B0E0AA0DBB1D8C93A2E606
:10012000B0E027D808F4E7CF88E48093640082E940
:100130008093E40084E28093640189E48093E40185
:100140008FEF809365008FEF8093E5008FEF8093B2
:1001500065018FE78093E50183E891E0A2E6B0E0D6
:100160008D939C93A2E6B0E00D911C91003052E07B
:10017000150710F009F00FC080E4A2E6B0E0AD90E2
:10018000BD90A3E6B0E0AA0DBB1D8C93A2E6B0E043
:10019000F0D708F4E7CF8FEF8093E3008FEF8093E1
:1001A00063018FEF8093E3018FE78093630278947C
:1001B000E2E6F7E149D84ED8B9D881E0809335031B
:1001C00081E08093360381E080933703E2E7F7E133
:1001D00050D886E08093350381E0809336038827EA
:1001E00080933703E8E8F7E144D887E0809335034C
:1001F00081E080933603882780933703EEE8F7E1A8
:1002000038D888E08093350381E0809336038827CF
:1002100080933703E4E9F7E12CD889D377DAA4E6B1
:10022000B2E0E0E3D0D76FDAA8E7B3E0AAD96EDA9C
:10023000A4E6B2E0E0E3C7D766DAA8E7B3E0A1D965
:10024000A5EEB2E089D74FEF50EE65EF75E0A5EE71
:10025000B2E00D911D912D913C91041715072607D1
:10026000370710F009F001C00AC000E010E020E0FC
:1002700030E0A5EEB2E00D931D932D933C9380E208
:10028000A4E6B2E0FFD8E4E6F2E09CE20AE037E060
:10029000A5E9B2E040DAA2EEB2E02C93A4E6B2E027
:1002A000CDD7D8D7A5E9B2E0C9D7ECE9F7E1CCD7EB
:1002B000A0EAB2E0C3D7CED7ABEAB2E0BFD7ECE951
:1002C000F7E1C2D7A6EBB2E0B9D7C4D7A1ECB2E050
:1002D000B5D7E4EAF7E1B8D7ACECB2E0AFD7BAD71C
:1002E000E8EAF7E1B1D7A7EDB2E0A8D7B3D7B2D724
:1002F000A0EAB2E0B5D9A3EEB2E00D931C9381E081
:1003000080936000009160000B3310F009F019C079
:10031000A0E6B0E0AD90BB24A3EFB2E0AA0DBB1DF8
:100320008C91A0E6B0E0AD90BB24A2EFB2E0AA0DA4
:10033000BB1D8C93A0E6B0E08C918F5F8C9308F48A
:10034000E1CF8091E30280932E0381E080936000EF
:10035000009160000C3310F009F006C2A0E6B0E096
:10036000AD90BB24A2EFB2E0AA0DBB1D0C910030F2
:1003700009F00CC000E010E020E030E5AFE2B3E0AF
:100380000D931D932D933C93B0C1AFC1093010F074
:1003900009F00CC000E010E020E038E5AFE2B3E087
:1003A0000D931D932D933C93A0C19FC1033110F079
:1003B00009F00CC000E010E020E03CE5AFE2B3E063
:1003C0000D931D932D933C9390C18FC10C3110F070
:1003D00009F00CC000E010E020E03EE5AFE2B3E041
:1003E0000D931D932D933C9380C17FC1063210F075
:1003F00009F00CC000E010E020E03FE5AFE2B3E020
:100400000D931D932D933C9370C16FC10F3210F06B
:1004100009F00CC000E010E020E83FE5AFE2B3E0F7
:100420000D931D932D933C9360C15FC1093310F070
:1004300009F00CC000E010E020EC3FE5AFE2B3E0D3
:100440000D931D932D933C9350C14FC1023410F076
:1004500009F00CC000E010E020EE3FE5AFE2B3E0B1
:100460000D931D932D933C9340C13FC10C3410F06C
:1004700009F00CC000E010E020EF3FE5AFE2B3E090
:100480000D931D932D933C9330C12FC1053510F072
:1004900009F00CC000E010E028EF3FE5AFE2B3E068
:1004A0000D931D932D933C9320C11FC10E3510F069
:1004B00009F00CC000E010E02CEF3FE5AFE2B3E044
:1004C0000D931D932D933C9310C10FC1083610F06E
:1004D00009F00CC000E010E02EEF3FE5AFE2B3E022
:1004E0000D931D932D933C9300C1FFC0013710F075
:1004F00009F00CC000E010E02FEF3FE5AFE2B3E001
:100500000D931D932D933C93F0C0EFC00B3710F06B
:1005100009F00CC000E010E82FEF3FE5AFE2B3E0D8
:100520000D931D932D933C93E0C0DFC0043810F071
:1005300009F00CC000E010EC2FEF3FE5AFE2B3E0B4
:100540000D931D932D933C93D0C0CFC00E3810F067
:1005500009F00CC000E010EE2FEF3FE5AFE2B3E092
:100560000D931D932D933C93C0C0BFC0073910F06D
:1005700009F00CC000E010EF2FEF3FE5AFE2B3E071
:100580000D931D932D933C93B0C0AFC0013A10F072
:1005900009F00CC000E018EF2FEF3FE5AFE2B3E049
:1005A0000D931D932D933C93A0C09FC00A3A10F069
:1005B00009F00CC000E01CEF2FEF3FE5AFE2B3E025
:1005C0000D931D932D933C9390C08FC0033B10F06F
:1005D00009F00CC000E01EEF2FEF3FE5AFE2B3E003
:1005E0000D931D932D933C9380C07FC00D3B10F065
:1005F00009F00CC000E01FEF2FEF3FE5AFE2B3E0E2
:100600000D931D932D933C9370C06FC0063C10F06A
:1006100009F00CC000E81FEF2FEF3FE5AFE2B3E0B9
:100620000D931D932D933C9360C05FC0003D10F06F
:1006300009F00CC000EC1FEF2FEF3FE5AFE2B3E095
:100640000D931D932D933C9350C04FC0093D10F066
:1006500009F00CC000EE1FEF2FEF3FE5AFE2B3E073
:100660000D931D932D933C9340C03FC0033E10F06B
:1006700009F00CC000EF1FEF2FEF3FE5AFE2B3E052
:100680000D931D932D933C9330C02FC00C3E10F062
:1006900009F00CC008EF1FEF2FEF3FE5AFE2B3E02A
:1006A0000D931D932D933C9320C01FC0063F10F067
:1006B00009F00CC00CEF1FEF2FEF3FE5AFE2B3E006
:1006C0000D931D932D933C9310C00FC00F3F10F05E
:1006D00009F00BC00EEF1FEF2FEF3FE5AFE2B3E0E5
:1006E0000D931D932D933C9300C00091600042E058
:1006F000049FA1E6B0E00C92A1E6B0E08C918E5F81
:100700008C9380912F03A1E6B0E0AD90BB24A3E6CB
:10071000B0E0AA0DBB1D8C9380913003A1E6B0E040
:10072000AD90BB24A3EEB0E0AA0DBB1D8C938091CD
:100730003103A1E6B0E0AD90BB24A3E6B1E0AA0D81
:10074000BB1D8C9380913203A1E6B0E0AD90BB2439
:10075000A3EEB1E0AA0DBB1D8C93A0E6B0E08C9196
:100760008F5F8C9308F4F4CDE2D0A7EDB2E0E2EB1A
:10077000F7E1B6D709F00BC0A3EEB2E00D911C91E2
:100780004CE350E087D6A3EEB2E00D931C9386E0D5
:100790008093350389E2809336038827809337035B
:1007A000E8EBF7E166D586E08093350388E4809333
:1007B0003603882780933703E8EBF7E15AD587E0C3
:1007C0008093350389E2809336038827809337032B
:1007D000E8EBF7E14ED588E08093350389E280931A
:1007E0003603882780933703E2ECF7E142D588E0AF
:1007F0008093350384E680933603882780933703FC
:10080000E2ECF7E136D5E5EEF2E0A9EEB2E0DAD6B9
:10081000E9EEF2E0A0EAB3E052D7E0EAF3E0A9EEB5
:10082000B2E01127222708E0332742D686E08093E2
:10083000350389E280933603882780933703E3EEFC
:10084000F2E0A0EAB3E0B9D60CD586E08093350398
:1008500088E480933603882780933703A9EEB2E0BB
:1008600002D587E08093350389E280933603882799
:1008700080933703A6EBB2E0F6D488E0809335038B
:1008800089E280933603882780933703ACECB2E08B
:10089000EAD488E08093350384E680933603882782
:1008A00080933703A7EDB2E0DED4C1CCF894FFCF3C
:1008B0000F921F922F923F924F925F927F92AF9230
:1008C000BF920F931F932F933F934F935F936F9319
:1008D0007F938F939F93AF93BF93CF93DF93EF93C8
:1008E000FF938FB78F938EEE95E89DBD8CBD85B33A
:1008F00091E0892785BB8F918FBFFF91EF91DF91A9
:10090000CF91BF91AF919F918F917F916F915F91A7
:100910004F913F912F911F910F91BF90AF907F907A
:100920005F904F903F902F901F900F90189581EB04
:10093000D7D480E1D5D480E0D3D481E090E0A2E6A2
:10094000B0E08D939C93A2E6B0E00D911C9100382D
:1009500050E0150710F009F00FC0A2E6B0E0AD902E
:10096000BD90A3E6B0E0AA0DBB1D8C91BCD4A2E65D
:10097000B0E0FFD308F4E7CF82EBB2D480E1B0D48B
:1009800080E0AED481E890E0A2E6B0E08D939C9345
:10099000A2E6B0E00D911C91003051E0150710F077
:1009A00009F00FC0A2E6B0E0AD90BD90A3E6B0E0C4
:1009B000AA0DBB1D8C9197D4A2E6B0E0DAD308F45F
:1009C000E7CF83EB8DD480E18BD480E089D481E0C4
:1009D00091E0A2E6B0E08D939C93A2E6B0E00D9189
:1009E0001C91003851E0150710F009F00FC0A2E685
:1009F000B0E0AD90BD90A3E6B0E0AA0DBB1D8C9118
:100A000072D4A2E6B0E0B5D308F4E7CF84EB68D4A3
:100A100080E166D480E064D481E891E0A2E6B0E0B1
:100A20008D939C93A2E6B0E00D911C91003052E0B2
:100A3000150710F009F00FC0A2E6B0E0AD90BD9030
:100A4000A3E6B0E0AA0DBB1D8C914DD4A2E6B0E0A8
:100A500090D308F4E7CF0895F894FFCF0108080277
:100A600000000000000000000000065F060000001B
:100A7000000703000703000000247E247E240000FA
:100A800000242B6A12000000006313086463000056
:100A90000036495620500000000007030000000007
:100AA00000003E41000000000000413E0000000048
:100AB00000083E1C3E0800000008083E0808000030
:100AC0000000E060000000000008080808080000BE
:100AD0000000606000000000002010080402000018
:100AE000003E5149453E00000000427F40000000AA
:100AF0000062514949460000002249494936000038
:100B0000001814127F100000002F494949310000DD
:100B1000003C4A494930000000017109050300000A
:100B2000003649494936000000064949291E00009F
:100B300000006C6C000000000000EC6C0000000085
:100B40000008142241000000002424242424000072
:100B500000004122140800000002015909060000AB
:100B6000003E415D551E0000007E1111117E000007
:100B7000007F494949360000003E414141220000C2
:100B8000007F4141413E0000007F4949494100004A
:100B9000007F090909010000003E4149497A00002F
:100BA000007F0808087F00000000417F410000002E
:100BB00000304040403F0000007F08142241000008
:100BC000007F404040400000007F0204027F0000A0
:100BD000007F0204087F0000003E4141413E0000CA
:100BE000007F090909060000003E4151215E000016
:100BF000007F0909196600000026494949320000B2
:100C00000001017F01010000003F4040403F000023
:100C1000001F2040201F0000003F403C403F0000DC
:100C20000063140814630000000708700807000040
:100C3000007149454300000000007F414100000071
:100C40000002040810200000000041417F00000065
:100C50000004020102040000808080808080808087
:100C600000000307000000000020545454780000E6
:100C7000007F4444443800000038444444280000C5
:100C800000384444447F00000038545454080000A5
:100C900000087E09090000000018A4A4A47C00003C
:100CA000007F0404780000000000007D4000000088
:100CB000004080847D000000007F10284400000078
:100CC0000000007F40000000007C04180478000051
:100CD000007C0404780000000038444444380000DC
:100CE00000FC4444443800000038444444FC000004
:100CF00000447844040800000008545454200000C4
:100D000000043E4424000000003C40207C00000021
:100D1000001C2040201C0000003C6030603C0000B3
:100D2000006C10106C000000009CA0603C000000F3
:100D3000006454544C00000000083E414100000093
:100D40000000007700000000000041413E08000064
:100D50000002010201000000003C2623263C0000A6
:100D6000001EA1E121120000003D40207D00000096
:100D7000003854545509000000205555557800009E
:100D80000020555455780000002055555478000037
:100D90000020575557780000001CA2E222140000E2
:100DA00000385555550800000038555455080000C6
:100DB00000385555540800000000017C4100000037
:100DC00000000279420000000000017C40000000A9
:100DD000007029242970000000782F252F7800004A
:100DE000007C5454554500000034547C5458000095
:100DF000007E097F49490000003845453900000060
:100E000000384544390000000039454438000000EE
:100E1000003C41217D000000003D41207C0000009D
:100E2000009CA1603D000000003D42423D000000EA
:100E3000003C41403D0000000018246624000000F2
:100E400000483E494962000000292A7C2A29000006
:100E5000007F0916781000000040887E090200001B
:100E600000205455557800000000007D410000002E
:100E70000038444539000000003C40217D0000005E
:100E8000007A090A71000000007A1122790000003E
:100E900000085555555E0000004E51514E000000AF
:100EA0000030484D40200000003C040404040000D1
:100EB00004040404041C00000017084C6A500000DD
:100EC000001708342A7800000000307D3000000050
:100ED00000081400081400000014080014080000A2
:100EE0004411441144110000AA55AA55AA55000006
:100EF000BBEEBBEEBBEE0000000000FF00000000F8
:100F0000080808FF000000000A0A0AFF00000000AD
:100F100008FF00FF0000000008F808F800000000CB
:100F20000A0A0AFE000000000AFB00FF00000000A1
:100F300000FF00FF000000000AFA02FE00000000AF
:100F40000A0B080F00000000080F080F0000000047
:100F50000A0A0A0F00000000080808F80000000054
:100F60000000000F080800000808080F080800002B
:100F7000080808F808080000000000FF0808000042
:100F80000808080808080000080808FF080800000A
:100F9000000000FF0A0A000000FF00FF0808000030
:100FA000000F080B0A0A000000FE02FA0A0A0000FD
:100FB0000A0B080B0A0A00000AFA02FA0A0A0000E1
:100FC00000FF00FB0A0A00000A0A0A0A0A0A0000D7
:100FD0000AFB00FB0A0A00000A0A0A0B0A0A0000C0
:100FE000080F080F080800000A0A0AFA0A0A000097
:100FF00008F808F808080000000F080F08080000AB
:101000000000000F0A0A0000000000FE0A0A0000AB
:1010100000F808F80808000008FF00FF08080000B2
:101020000A0A0AFB0A0A00000808080F000000006C
:10103000000000F808080000FFFFFFFFFFFF0000AE
:10104000F0F0F0F0F0F00000FFFFFF000000000003
:10105000000000FFFFFF00000F0F0F0F0F0F000039
:10106000001824241824000000FE4A4A340000001E
:10107000007F01010300000000027E027E020000EA
:101080000063554963000000001824241C0400007C
:1010900000FC20201C000000000804780400000070
:1010A0000008557755080000003E49493E00000001
:1010B000004C7202724C00000022555930000000B2
:1010C00000182418241800000018247E241800009A
:1010D000001C2A2A2A000000003C02023C000000FA
:1010E000002A2A2A2A0000000000242E24000000E2
:1010F00000514A4A4400000000444A4A510000009E
:10110000000000FC020400000020403F000000003E
:101110000008082A08080000002412241200000019
:101120000006090906000000000018180000000071
:1011300000000800000000000030403E02020000F5
:1011400000010E010E00000000090D0A0000000061
:10115000003C3C3C3C0000000D911D912D913C91C8
:101160000F5F1F4F2F4F3F4F3C932E931E930E93B5
:101170000895ED91FC91EF5FFF4FFC93EE9308957E
:1011800004D088D100FC0CD008950024E89457FFC7
:1011900002C009D0689400F80BD010F8012408951B
:1011A00002D009D00895509540954F5F5F4F089544
:1011B000E89417FF0895009510950F5F1F4F6894EE
:1011C0000895A0EAB3E014D08D30E9F38A3039F005
:1011D000EE23C9F38D93EA9563FE3FD0F4CF63FC11
:1011E00004C08DE03AD08AE038D088278C930895E7
:1011F0000F929F93AF93BF937F9380917A0388233D
:10120000E1F3F89480917A038A9580937A03909120
:101210007803A8E3B3E0A90F0024B01D8C91939547
:10122000903409F499279093780378947F91BF9133
:10123000AF919F910F900895A0EAB3E08D9188231C
:1012400011F00BD0FBCF08952FD1802D11F005D0D8
:10125000FBCF08958DE001D08AE05D9BFECF8CB975
:101260000895A0EAB3E08D91882311F008D0FBCF58
:1012700008951AD1802D11F002D0FBCF089567C0D8
:101280003197F1F70895689462F80895E89462F848
:101290000895EF93FF93EE27E82BE92B31F0E0ED73
:1012A000F7E03197F1F70197D1F7FF91EF910895AA
:1012B000959882E39927EDDF959AC598949AE0ED89
:1012C000F2E11FE0F1D0802D0BD01A95D9F70895E7
:1012D000E240A1C0A6A22FF800278116AC00AF0003
:1012E0007F93979802C07F93979A949898E0880F7D
:1012F00010F4C39A02C0C3980000C5980000000013
:101300000000000000000000000000000000C59A7E
:1013100000000000000000000000000000000000CD
:1013200000009A9521F7949A7F91089500E080EB50
:10133000800FD6DF80E1D4DF8827D2DF14E888274A
:10134000D2DF1A95E1F70395083089F70895EF93F6
:10135000FF93509135035F9370903603E091330310
:10136000F0913403A1D0202D9FD0302D9DD0002DA1
:101370009BD0602D8052482FA7D1E40FF51FCC24BD
:101380001124E22E603051F1DD24DA94CD2CFF24BB
:10139000032F8AD021F00A95E00FF11D03C0F394CA
:1013A0000A95B9F7FD1408F4DF2CEA9481F7E22ED0
:1013B000FF24032F3197C895002021F00A95E01BE8
:1013C000F10903C0F3940A95A9F7FC1408F4CF2C93
:1013D000EA9471F7D31611F4D62ECC24709236030A
:1013E000732F7C19409136035091350339D060300A
:1013F00039F0DD2029F05D2D57D05A95E9F77D1998
:1014000053D0802D50913703552309F080956BDF21
:10141000509136035395509336037A9589F7EC0D26
:10142000F11D603079F050913703762F88275523CE
:1014300009F0809558DF7A95C9F750913603560F19
:1014400050933603509135035395509335032A95A5
:1014500009F0C4CF5F9150933503FF91EF91089548
:101460004A955A9580EB850F3BDF842F82958F70CC
:10147000806136DF842F8F7033CF019111912191DC
:1014800030810895FD019D91981709F0919399235A
:10149000D1F708950F92B801469F8001479F100D24
:1014A000569F100D0F900895C8953196002008950D
:1014B0002E2E3F2E992781918D3209F09395882306
:1014C000D1F79A95E22DF32D112361F0091718F049
:1014D00011F0101B01C0191B28F021F080E28D9340
:1014E0001A95E9F780818D3219F48D93319604C0F5
:1014F000222311F08BE28D93091738F031F0091B8C
:1015000021F080E38D930A95E9F781918D938823EB
:10151000E1F7332351F0EA2FFB2F319633958E916B
:1015200082933A95E1F78EE28C9308957F930F931F
:10153000AF93BF938F939F938FB78F9380917A03CD
:1015400000E4081B19F49CB19EDE12C000917903DF
:10155000A8E3B3E077279CB1A00FB71F9C938395B6
:1015600080937A030395003409F4002700937903EC
:101570008F918FBF9F918F91BF91AF910F917F916D
:1015800018956FB7F894882793E08D939A95E9F7AB
:101590006FBF0895040F151F261F371F0895000FF2
:1015A000111F221F331F0895009510952095309527
:1015B0000F5F1F4F2F4F3F4F0895019110810DC0B6
:1015C0005CDF0DC05ADF10C00191108117FF05C00C
:1015D0003FEF2FEF04C0008111272227332737FF69
:1015E00003C0E2DF8DE28D93CF92DF92EF92AA24C7
:1015F000BB24CC24DD24EE2440E2EAE0FF2755E0C2
:1016000093E38081890F87FD9F7083FD907F891B05
:1016100081935A95A9F7C3DFAA1CBB1CCC1CDD1C07
:10162000EE1C4A9551F7E894EFE0FF2782910BD02A
:10163000EB30E0F71EF068948A2D09D04D93EF90BF
:10164000DF90CF900895982F829501D0892F8F70C9
:10165000805D26F0803309F4089568948D93089591
:1016600000271127222733271DD08A3328F48033FF
:1016700018F005D015D0F9CF0EF496CF0895805309
:101680008F93402F512F622F732F89DF88DF82DFE6
:1016900086DF8F919927080F191F291F391F089579
:1016A0008D910895E894FCDF8032E9F38B32D9F311
:1016B0008930C9F38D3211F46894F2CF0895819185
:1016C0008D938823E1F70895FF935527F8E0469519
:1016D00008F4500F57954795FA95D1F7FF91089563
:1016E000689401C0E894AF93BF938D9116F09191E7
:1016F00002C0DADE902D891718F011F48823A9F7BB
:10170000BF91AF910895E89463F80895689463F8E1
:101710000895689401C0E8942227102F231709F434
:1017200008951EF4C1DE802D01C08191803081F0CA
:10173000891741F070E08D931A9599F7239571E020
:101740001D93EBCF01D0E9CF703011F077270895CA
:10175000772331F42395882713958D931A95E9F70C
:10176000089550726F6772616D6D20737461727449
:1017700000002A204D794765696765726C652056BF
:10178000312E3031202A00004350533A000043509C
:101790004D3A00007553762F683A00002020202033
:1017A0003A200000203A20004D6F64652020203A46
:1017B0002000494E535400002020202020202020CB
:0817C0000000202020200000A1
:00000001FF
